:02000000912E3F
:100D2200F001F101F201F301F401F50183012D2F2C
:100D3200831203130515A730F2000030F300730885
:100D42007204031DA52EA62EA82E202F202F8F3031
:100D5200831203139F000330F7009730F600F60B5F
:100D6200B02EF70BB02EB52EB62E831203139F189A
:100D7200BB2EBC2EB62EBD2E1E080339F600F7017F
:100D82007608F700F601831603131E087607F000B3
:100D92000030031801307707F100003071020A3089
:100DA200031970020318D62ED72E0B2FD030FB005A
:100DB2000730FC007C087B04031DE02EE12EE32EAD
:100DC2000B2F0B2F831203138617000083120313BA
:100DD20086130730F6007608F400F408031DF22E9D
:100DE200F32EF52EFD2EFD2E0130F402F408031D24
:100DF200FB2EFC2EF52EFD2E0130FB020030031CD3
:100E0200FC03FC027C087B04031D082F092FE32E40
:100E12000B2F0B2F0330F7009730F600F60B0F2F36
:100E2200F70B0F2F142F0130F2020030031CF303D3
:100E3200F30273087204031D1F2F202FA82E8312A2
:100E4200031305110330F7009730F600F60B272F36
:100E5200F70B272F2C2F08008B1383120313850106
:100E6200860187013B3083160313850070308600AC
:100E7200CE30870004309100930170308F008030B3
:100E8200831203179C0080309D00103083160313D9
:100E92009F00831203130515F430FB000130FC00A0
:100EA2007C087B04031D562F572F592F792F792F3A
:100EB2000330F9009730F800F80B5D2FF90B5D2F26
:100EC200622F831203138617000083120313861303
:100ED20000000000000000000130FB020030031C93
:100EE200FC03FC027C087B04031D782F792F592F09
:100EF200831203130511003087180130F8007808B7
:100F0200F5000030831203138718013075060319A8
:100F12008B2F8C2F822F003087180130F800780831
:100F2200F5003430F900F130F800F80B962FF90B88
:100F3200962F9B2F0A30FB000030FC0000308312FA
:100F42000313871801307506031DA82FA92FE62F5A
:100F5200DA2FDA2F05150330FA000830F90078305D
:100F6200F800F80BB22FF90BB22FFA0BB22F831243
:100F7200031305110330FA000830F9007830F80045
:100F8200F80BC12FF90BC12FFA0BC12F0130FB0255
:100F92000030031CFC03FC02FF307C06031DD32F30
:100FA200FF307B06031DD62FD72FDA2FE62FE62F31
:100FB200DA2F0030831203138718013075060319E4
:100FC200E32FE42FAB2FE62FE62F99260030831272
:100FD200031387180130F8007808F5000230FA0090
:100FE2000430F900BA30F800F80BF52FF90BF52FA1
:0E0FF200FA0BF52F6400822F822F822F002829
:02400E00E4309C
:00000001FF
